:100000000C94CA050C9443310C9411060C941106FF
:100010000C9411060C9411060C9411060C94110604
:100020000C9411060C9411060C94101A0C94CC1913
:100030000C944F1C0C9411060C9411060C94110690
:100040000C9411060C9411060C9411060C941106D4
:100050000C9411060C942B1C0C9411060C94110694
:100060000C9411060C9411060C9411060C941106B4
:100070000C9411060C9411060C9411060C941106A4
:100080000C9411060C9411060C9411060C94110694
:100090000C9411060C9411060C9411060C94110684
:1000A0000C9411060C9411060C9411060631FF09EC
:1000B00074A1010975150026FF00952075088102BD
:1000C0000976150026FF00952075089102C00501EC
:1000D0000980A101850319012AB700150126B7007F
:1000E000950175108100C0050C0901A10185041955
:1000F000012AA002150126A002950175108100C0F9
:100100000660FF0961A1010962150026FF00952024
:10011000750881020963150026FF00952075089176
:1001200002C005010906A101050719E029E715002C
:100130002501950875018102950175088101050762
:10014000190029FF150026FF009506750881000596
:10015000081901290595057501910295017503910D
:1001600001C00001010101010101010102020202BD
:100170000202020202030303030303030304040451
:10018000040404040505050505060606060607071A
:1001900007070708080808090909090A0A0A0B0BD2
:1001A0000B0C0C0C0D0D0D0E0E0E0F0F0F10101171
:1001B00011111212131314141515161617171818F7
:1001C00019191A1A1B1B1C1D1D1E1E1F202021225F
:1001D00022232424252626272829292A2B2C2D2DA5
:1001E0002E2F30313232333435363738393A3B3CC2
:1001F0003D3E3F404142434445464748494A4C4DB5
:100200004E4F50515354555658595A5B5D5E5F617D
:100210006264656668696B6C6D6F70727375777810
:100220007A7B7D7E8082838587888A8C8E8F91936E
:100230009596989A9C9EA0A2A3A5A7A9ABADAFB195
:10024000B3B5B7BABCBEC0C2C4C6C9CBCDCFD1D47A
:10025000D6D8DBDDDFE2E4E7E9EBEEF0F3F5F8FA20
:10026000FDFF7267626C69676874206D6F6465205A
:100270005B4E4F454550524F4D5D3A2025750A0063
:100280007267626C69676874206D6F6465205B4596
:100290004550524F4D5D3A2025750A007267626CD9
:1002A000696768742064697361626C65205B4E4F96
:1002B000454550524F4D5D3A207267626C696768E0
:1002C000745F636F6E6669672E656E61626C652030
:1002D0003D2025750A007267626C69676874207337
:1002E000657420687376205B4E4F454550524F4DE4
:1002F0005D3A2025752C25752C25750A00726762DC
:100300006C696768742073657420687376205B4538
:100310004550524F4D5D3A2025752C25752C25757D
:100320000A007267626C69676874207261696E6244
:100330006F7720736574206873763A2025642C25C6
:10034000642C25642C25750A00FFAA7F554072672E
:10035000626C696768742074696D657220656E618E
:10036000626C65642E0A007267626C69676874204B
:1003700074696D65722064697361626C652E0A0030
:100380002223252628292A2C2D2F303233353638A2
:100390003A3B3D3E4042434547494A4C4E505153FB
:1003A0005557595A5C5E6062646668696B6D6F711F
:1003B000737577797B7D7F81838587898A8C8E9021
:1003C000929496989A9C9E9FA1A3A5A7A8AAACAE2A
:1003D000AFB1B3B4B6B8B9BBBCBEBFC1C2C3C5C66A
:1003E000C7C9CACBCCCDCED0D1D2D2D3D4D5D6D713
:1003F000D7D8D9D9DADADBDBDBDCDCDCDCDCDDDD51
:10040000DDDDDCDCDCDCDCDBDBDBDADAD9D9D8D740
:10041000D7D6D5D4D3D2D2D1D0CECDCCCBCAC9C7E2
:10042000C6C5C3C2C1BFBEBCBBB9B8B6B4B3B1AF19
:10043000AEACAAA8A7A5A3A19F9E9C9A98969492B9
:10044000908E8C8A89878583817F7D7B7977757390
:10045000716F6D6B6968666462605E5C5A5957556E
:100460005351504E4C4A4947454342403E3D3B3A2A
:100470003836353332302F2D2C2A292826252322B1
:1004800029001E001F002000210022002B00140064
:100490001A00080015001700E0000400160007000D
:1004A00009000A00E1001D001B00060019000500FC
:1004B00000000000E300105F28004A002A00270027
:1004C00026002500240023004C00130012000C001D
:1004D00018001C00340033000F000E000D000B004C
:1004E000E500380037003600100011000000000061
:1004F000E200115F2C004D0035021E021F02200297
:1005000021022202005C1E001F00200021002200A8
:100510004C00010050004F0052002F00C05C010051
:100520000100010051002F02000000000100010045
:100530004C0026022A00270226022502240223025A
:1005400001002700260025002400230031022E028E
:100550005E005D005C00300001002D005B005A0071
:100560005900300200000000620001004C00270228
:1005700045003A003B003C003D003E00C25C1E02CC
:100580001F02200221022202C35CAC00AB00A900C2
:100590004B002D02A800AD00AE00AA004E002D00B9
:1005A0000000000001000100010026024400430099
:1005B0004200410040003F000100270226022502C0
:1005C000240223023100C95CC75CC55C4A002E00CE
:1005D0000100CA5CC85CC65C4D002E020000000031
:1005E0000100010001000100010001000100010003
:1005F00001000100010001000100010001000100F3
:1006000001000100010001000100010001000100E2
:1006100001000100010001000000000001000100D4
:1006200001000100010001000100010001000100C2
:1006300001000100010001000100010001000100B2
:1006400001000100010001000100010001000100A2
:100650000100010000000000010001000100010094
:10066000000000000000000000000000000000008A
:10067000000000000000000000000000000000007A
:10068000000000007E0F00D4FFFFFFC700000078CD
:1006900000000000000000002A2B280000000000DD
:1006A0000000000000000000000000290000000021
:1006B0002C1E3420212224342627252E362D37388F
:1006C000271E1F202122232425263333362E373898
:1006D0001F0405060708090A0B0C0D0E0F10111256
:1006E000131415161718191A1B1C1D2F3130232D22
:1006F000350405060708090A0B0C0D0E0F10111220
:10070000131415161718191A1B1C1D2F3130354CD0
:100710006261636B6C6967687420646563726561AC
:1007200073653A2025750A006261636B6C696768BE
:100730007420696E6372656173653A2025750A00DD
:100740006261636B6C696768742064697361626C71
:10075000650A006261636B6C6967687420656E612D
:10076000626C650A006261636B6C6967687420740F
:100770006F67676C653A2025750A006261636B6C70
:100780006967687420737465703A2025750A007271
:1007900067626C696768742064697361626C652064
:1007A0005B454550524F4D5D3A207267626C6967F8
:1007B00068745F636F6E6669672E656E61626C65F3
:1007C000203D2025750A007267626C696768742095
:1007D000656E61626C65205B454550524F4D5D3AD8
:1007E000207267626C696768745F636F6E666967C1
:1007F0002E656E61626C65203D2025750A0072676A
:10080000626C6967687420746F67676C65205B450C
:100810004550524F4D5D3A207267626C696768744B
:100820005F636F6E6669672E656E61626C65203D01
:100830002025750A0044454255473A206469736192
:10084000626C65642E0A0044454255473A20656E45
:1008500061626C65642E0A004F6E6573686F743A4E
:10086000206163746976653A2025640A000A0025D0
:1008700030325820006B6579626F6172645F726517
:10088000706F72743A20007267626C696768745F97
:10089000636F6E6669672E7370656564203D202501
:1008A000640A007267626C696768745F636F6E6682
:1008B00069672E76616C203D2025640A00726762AC
:1008C0006C696768745F636F6E6669672E736174C5
:1008D000203D2025640A007267626C696768745F56
:1008E000636F6E6669672E687565203D2025640A12
:1008F000007267686C696768745F636F6E666967CA
:100900002E6D6F6465203D2025640A007267626C5D
:10091000696768745F636F6E6669672E656E616292
:100920006C65203D2025640A007267626C69676807
:10093000745F636F6E66696720454550524F4D3A4C
:100940000A007267626C696768745F696E69742017
:100950007267626C696768745F636F6E6669672E41
:100960006D6F6465203D20302E20577269746520BC
:1009700064656661756C742076616C75657320744E
:100980006F20454550524F4D2E0A007267626C69C8
:100990006768745F696E6974206565636F6E666908
:1009A00067206973206E6F7420656E61626C656488
:1009B0002E0A007267626C696768745F696E697499
:1009C000207374617274210A007267626C696768CF
:1009D000745F696E69742063616C6C65642E0A00D3
:1009E0000A0025303862003A200025303258000ACB
:1009F000722F632030313233343536370A00726754
:100A0000626C6967687420616E696D6174696F6E8C
:100A1000207469636B207265706F727420746F202C
:100A2000736C6176650A0000047F3F1F64321464B2
:100A30003214783C1E1E140A050A00253032580074
:100A40006B6579626F6172645F7365745F6C656416
:100A50003A20007267626C6967687420656E616233
:100A60006C65205B4E4F454550524F4D5D3A2072AC
:100A700067626C696768745F636F6E6669672E652D
:100A80006E61626C65203D2025750A007267626C9C
:100A90006967687420736574207370656564205B92
:100AA0004E4F454550524F4D5D3A2025750A005B2B
:100AB000735D004B6579626F61726420737461725B
:100AC000742E0A005B435D005B445D005B535D0078
:100AD0005B575D005B525D0009027B00040100A0D2
:100AE000FA090400000103010100092111010001BC
:100AF0002240000705810308000A090401000203DF
:100B000000000009211101000122220007058203D3
:100B1000200001070503032000010904020001036E
:100B200000000009211101000122320007058403A1
:100B300020000A090403000203000000092111013A
:100B40000001222200070585032000010705050397
:100B5000200001120110010000000810CB565200C5
:100B600005010200011803490072006900730020AA
:100B7000005200650076002E002000350000000EB7
:100B8000034B0065006500620069006F000000040F
:100B90000309040011241FBECFEFDAE0DEBFCDBF92
:100BA00004B603FE27C08091E7029091E802A0916D
:100BB000E902B091EA028730904BA740B04BD1F4E4
:100BC0001092E7021092E8021092E9021092EA02F3
:100BD00014BE84B7877F84BF0FB6F894A895809120
:100BE0006000886180936000109260000FBEE0E0BA
:100BF000F8E3099511E0A0E0B1E0E0E2F7E602C019
:100C000005900D92A23CB107D9F722E0A2ECB1E029
:100C100001C01D92A73EB207E1F70E946C280C9418
:100C200057330C940000FF93EF93E091C201F091D1
:100C3000C301309709F00995EF91FF910895FC01E8
:100C40008591803011F0EFDFFBCF0895FF27E0E2C0
:100C500030E247FF0CC0419597FF09C0EDE2609577
:100C6000709580959095611D711D811D911D27FFC7
:100C700002C0219530E350E2AA27660F771F881F34
:100C8000991FAA1FA41710F0A41B63955A95A9F7E2
:100C9000AA3008F0A95FA05DAF93F39561157105C7
:100CA0008105910541F7ED3211F4EF93F395F217B9
:100CB00018F43F93F395FBCF8F91B5DFFA95E1F7E9
:100CC0000895E991F9918591803021F0853219F0EC
:100CD000AADFF9CF089520E0E89455915532C1F389
:100CE000503311F4689455915A3348F4505390F3AB
:100CF000220F022E220F220F200D250FF4CF0EF40B
:100D0000219589919991533619F3533729F1533528
:100D100059F1BC0188279927E8945C3621F4899120
:100D2000999168945591543639F446EF7EF077FFE7
:100D30000DC08FEF9FEF0AC055374AE039F05835A4
:100D400040E121F0523642E009F00895FF93EF931D
:100D50007DDFEF91FF91B7CFFF93EF93FC0181917E
:100D60008030B9F360DFFBCFFF93EF9368DFF1CF03
:100D7000DF93CF93CDB7DEB72596A3DFCF91DF9179
:100D80000895E8EDF0E080818E7F80831092E2008C
:100D90001092DA001092E100A0EEB0E08C91816038
:100DA0008C9380818F77808319BCA7EDB0E08C9104
:100DB0008E7F8C9380818F7E80831092AD02089508
:100DC0002091E4003091E50095E6A9012091EC0026
:100DD000822F817020FF06C08091E80080FF06C04E
:100DE00080E008952091E80022FD1AC08091BA02A7
:100DF000882389F0853089F08091EB0085FD0FC054
:100E00002091E4003091E50042175307F9F2915028
:100E1000E1F684E0089582E0089583E0089581E09A
:100E20000895EF92FF920F931F93CF937C018B0154
:100E30000E94E006C82F811117C08091E80085FD4F
:100E40000BC08091E8008E778093E8000E94E00656
:100E5000882399F3C82F08C0F70181917F018093FF
:100E6000F1000150110949F78C2FCF911F910F917B
:100E7000FF90EF9008958091BC0287FF13C080918E
:100E8000E80082FF06C08091E8008B778093E8003D
:100E900004C08091BA028111F2CF08958091BA0204
:100EA0008823D9F38091E80080FFF8CF8091E80093
:100EB0008E77ECCF982F9093E900242F762F50E077
:100EC000891731F07091EC002091ED005091F00005
:100ED00021FD07C09F5F973071F78093E90081E0A3
:100EE00008953091EB003E7F3093EB003091ED00A0
:100EF0003D7F3093ED003091EB0031603093EB009B
:100F00007093EC002093ED005093F0002091EE00E0
:100F100027FDE0CF80E00895CF92DF92EF92FF921D
:100F20000F931F93CF93DF93C8EDD0E088818F7E1E
:100F30008883E7EDF0E080818160808384E082BF78
:100F400081E08093AD0288818E7F888302EE10E07D
:100F5000F80110821092DA0081EEC82ED12CF60131
:100F6000108288818F7788838881806888838881D0
:100F70008F7D888319BC1092BA021092BB02109226
:100F8000B9021092B80290EEE92EF12CF70180819F
:100F90008B7F808388818160888342E060E080E08D
:100FA0000E945A07F60180818E7F8083F80180813C
:100FB00081608083808188608083F70180818E7F5B
:100FC0008083888180618883DF91CF911F910F9109
:100FD000FF90EF90DF90CF900895FC018091C202C6
:100FE0009091C30286179707A0F06115710529F447
:100FF0009091E8009E779093E80090E0611571056C
:1010000051F4911108C08091E80082FF34C080E063
:101010000895BC01F2CF8091BA028823C1F18530D6
:10102000C1F18091E80083FD30C08091E80082FD2D
:10103000EACF8091E80080FFE1CF8091F30020911A
:10104000F200382F6115710519F02830310558F07C
:1010500091E02830310509F090E02091E8002E77EA
:101060002093E800CBCF81918093F100615071090A
:101070002F5F3F4FE7CF8091BA02882341F0853040
:1010800041F08091E80083FFBECF81E0089582E0C7
:10109000089583E00895089508958091AF0208951A
:1010A0002FB7F8946091C4027091C5028091C60276
:1010B0009091C7022FBF08952FB7F8948091C40272
:1010C0009091C502A091C602B091C7022FBF0895AA
:1010D000809161028111109261020895E6ECF1E0C5
:1010E0009191891303C0DF0111971C9291E0EC3CB0
:1010F000F907B1F70895A6ECB1E0EFEF90E02D917C
:10110000821751F0EF3F19F4211101C0E92F9F5FC1
:101110009630A9F7EF3F09F408950E2E000CFF0B4F
:10112000EC53FE4F82830895E92FEE0FE90FEE0F87
:101130008E0F982F977086958695869525E0829FCD
:10114000F0011124EB5CFD4F50E040E080E0219184
:1011500030E0092E02C0369527950A94E2F72170F7
:101160003327042E01C0220F0A94EAF7822B4F5F27
:101170005F4F4530510559F70895E92FEE0FE90FFC
:10118000EE0F8E0F982F977041E001C0440F9A9593
:10119000EAF786958695869595E0899FF00111245A
:1011A000EB5CFD4F30E020E070E05191DF011197E2
:1011B000CB01022E02C0969587950A94E2F78170C2
:1011C00081958527842385278C932F5F3F4F25307A
:1011D000310559F7089580913402909103029813D4
:1011E00001C008958F5F8770FACF0C94500820914A
:1011F000FA013091FB012817390771F09093FB0138
:101200008093FA01E0917B02F0917C02309721F00B
:101210000084F185E02D099408952091F801309122
:10122000F9012817390771F09093F9018093F801BB
:10123000E0917B02F0917C02309721F00680F781EB
:10124000E02D09940895E0917B02F0917C023097A3
:1012500021F00190F081E02D099480E00895FA01D9
:10126000811101C0FB01099480919C02982F9E7FFF
:1012700029F48170826080939C0208958A34E8F397
:1012800081708864F8CFAF92BF92DF92EF92FF92A5
:101290000F931F93CF93DF93082F162FE901E42FAD
:1012A000F0E0EE59FE4F611110C0E4915E2F4E2F19
:1012B0004983E8835A83DF91CF911F910F91FF906B
:1012C000EF90DF90BF90AF900895E62EF12C4491FF
:1012D000D42EE42FF0E026E0829FC00111242FEFEE
:1012E00030E0B9010E947A32802F90E0880F991F78
:1012F00055E5569FD001579FB00D11248A1B9B0BBB
:10130000982F990F890F5901AE18BF08AE9ED001D2
:10131000AF9EB00DBE9EB00D11245B2F189F8001B3
:101320001124012F11275901A01AB10AAE9E800184
:10133000AF9E100DBE9E100D11245901A81AB108C0
:10134000AE9CC001AF9C900DBE9C900D1124892FC6
:101350009927281B390B2E9FC0012F9F900D3E9F70
:10136000900D1124E92F62307105A1F050F4611540
:10137000710509F49DCF6130710581F0EB2F512F7C
:1013800097CF6430710569F080F06630710509F41B
:101390008FCFF4CFE42F4B2F592F8ACFE42F412F3B
:1013A00087CFEB2F542F492F83CF4B2F5D2DE12F6C
:1013B0007FCFF894E82FE295EF70F0E031A1282F6D
:1013C0002F7081E090E001C0880F2A95EAF7982FEE
:1013D0009095932391A392A1892B82A37894089549
:1013E00090916B0292FF06C0282F28712830F9F4E3
:1013F000877F846093FF06C0282F28712831F1F47D
:10140000877E846120916C0220FF06C0382F3871DE
:101410003830D9F4877F816021FF06C0282F2871DA
:101420002831D1F4877E816194FD877E0895282F2D
:1014300024712430F9F68B7F8860DCCF282F24714B
:10144000243101F78B7E8861DDCF382F3171313047
:1014500019F78E7F8860E0CF282F2171213121F785
:101460008E7E8861E1CF829590E09C01220F331F30
:10147000220F331F2C7C95958795959587958373BF
:10148000282B30E0C901880F991F8A7A3595279556
:101490002575822B0895CF9384E090E00E9402335B
:1014A000C82F82E290E00E940233982F8C2FCF91B8
:1014B00008950F931F93CF93DF93C42FD0E0CC0FE9
:1014C000DD1F2CE0629FC00DD11D112438E7839FE2
:1014D000C00DD11D1124CE0187960E940233082F22
:1014E00010E0102F0027CE0188960E940233980149
:1014F000282BC901DF91CF911F910F910895462F9D
:10150000843038F47A3028F4663018F4672F0C945D
:10151000590A90E080E00895CF93DF930E947F0AFC
:10152000EC0182389105A9F1D8F58133910509F4D0
:1015300096C048F58932910509F48AC08A9709F462
:1015400095C0C11522E5D20708F0B6C0C11531E536
:10155000D30708F026C1C83ED10508F09CC0C13EA3
:10156000D10560F5C83AD10508F087C0C53AD10564
:1015700008F0EFC0C130D10509F12097F9F0C4306F
:10158000D105E0F440C08533910509F45AC0C997EC
:10159000C1F680916B02837089F0C0EED0E00EC07E
:1015A000833E910599F170F4803E910501F1823EF0
:1015B000910539F680916B0282FD21C0CE01DF9149
:1015C000CF910895863E910561F1873E910571F1B5
:1015D000843E910509F0B5CF80916C0281FFEECF7A
:1015E00080916B02C7EED0E084FD0DC0E7CF809103
:1015F0006B0280FD07C190916C0290FFDFCFC3EEBC
:10160000D0E084FFDBCFD0E0C0E0D8CF80916B0288
:1016100082FDFBC090916C0290FDBFCF84FFCECFC6
:10162000F2CF80916B0283FDDDCFC8CF80916B023A
:1016300083FDEEC090916C0291FFF0CFC4EED0E03C
:10164000BDCF80916B0285FFB9CFC9E2D0E0B6CFA4
:1016500080916B0285FFB2CFC5E3D0E0AFCF809120
:101660006B0286FFABCFCAE2D0E0A8CF80916B02BD
:1016700086FFA4CFC1E3D0E0A1CFCF3BD10518F6C0
:10168000C85AD0E0CC0FDD1FC159DE4F0990D88178
:10169000C02DD46493CFC11540E5D40708F064C0D1
:1016A000C11580E4D80708F05CC0CE019A95811579
:1016B0009F4108F483CFA7CFC11536E5D30718F5AE
:1016C000C11545E5D40708F084C0C11584E5D807E5
:1016D00008F07AC09C2F969596959E01237033272B
:1016E000C115D34508F462C0C1E0D0E002C0CC0F00
:1016F000DD1F2A95E2F730E2939FC0011124C82B29
:10170000D92BDA685BCFC1158AE5D80778F4C11503
:1017100099E5D90708F068C0C11528E5D20708F493
:1017200072CFDC2FCC27C06FD06A48CFCE01905645
:101730008115904208F067CF8D2F8F710E94F009BC
:1017400090E0982F882788279F719C012C2BE90116
:1017500049C0C55AD0E0C459DE4FC881D0E0D0643A
:101760002DCFDF70D06A2ACFCE01E4E09695879521
:10177000EA95E1F783702C2F26952695237040E299
:10178000249F90011124382B8C2F8370C1E0D0E06E
:1017900002C0CC0FDD1F8A95E2F7C22BD32BDC6889
:1017A0000DCFDC2FCC27C16FD06A08CFC1E0D0E0CD
:1017B00002C0CC0FDD1F2A95E2F720E2929FC00104
:1017C0001124C82BD92BEBCFDC2FCC27C46FD06AC8
:1017D000F5CE8C2F0E94F009C82FD0E0DC2FCC274B
:1017E000CC27DF71D062EACE8C2F8F700E94F00977
:1017F00034E0D695C7953A95E1F7CF709C2FEC0170
:10180000D069DCCEC9E3D0E0D9CEC2EED0E0D6CEEE
:10181000C6EED0E0D3CEBF92CF92DF92EF92FF928E
:101820000F931F93CF93DF938C01C090CB02D09086
:10183000CC02E090CD02F090CE02809162029091B5
:101840006302A0916402B0916502C82AD92AEA2AEB
:10185000FB2ACFE1D0E0BC2ED701C6010C2E04C07C
:10186000B695A795979587950A94D2F780FD0EC0F7
:10187000219788F7B12C8B2DDF91CF911F910F917C
:10188000FF90EF90DF90CF90BF900895B8018C2F1C
:101890000E948C0A019761F3EECFCF93DF93EC01A6
:1018A0000E940B0CBE01DF91CF910C948C0A0E9418
:1018B0004D0C292F2F7092959F7092509E3078F486
:1018C000E92FF0E0E75AFC4C0C94C432803F19F049
:1018D00020F4883E20F481E00895843FE1F380E025
:1018E0000895883EC0F3813FD1F7F5CF822F8695CA
:1018F0008695869508956F927F928F929F92AF9270
:10190000BF92CF92DF92EF92FF920F931F93CF93EC
:10191000DF9380E8C82E84E0D82E9BEAE92EF12CD4
:10192000E701C857D10936011BC0F5018590949095
:10193000692DC8010E941633682DC80101960E94C6
:10194000163382E0A80EB11C0E5F1F4FC017D107DF
:1019500061F78CE0680E711C2C96CE15DF0529F01E
:101960008E010C5011095301E0CF7E0188E7E80E8B
:10197000F11C88E7C80ED11C8BE8E81682E0F80657
:1019800079F6DF91CF911F910F91FF90EF90DF904B
:10199000CF90BF90AF909F908F907F906F90089561
:1019A000CF93DF93C7E0D2E060E0CE010E94163310
:1019B0002196C11584E0D807B9F7DF91CF9108953A
:1019C000682F86E090E00C941633EF92FF920F930D
:1019D0001F93CF93DF938091600290915F02892BD8
:1019E00090915E02892B8093C401909161029923AA
:1019F00091F0892B8093C40120E086EC91E0FC01FA
:101A00003191CF0131112F5FF1E08C3C9F07B9F785
:101A100021110E946808E0917B02F0917C023097CE
:101A2000C9F10280F381E02D84EC91E00995809169
:101A30009B0282FF2FC080FF04C085E798E00E94D0
:101A40001F06C4ECD1E08CECE82E81E0F82E0FE606
:101A500018E080919B0280FF0BC088811F928F93BA
:101A60001F930F930E94B8060F900F900F900F9046
:101A70002196EC16FD0669F780919B0280FF0AC053
:101A80008DE698E0DF91CF911F910F91FF90EF903D
:101A90000C941F06DF91CF911F910F91FF90EF9053
:101AA000089590E080E00E940D0990E080E00E949F
:101AB000F70810925F0210925E020C94E50C60939E
:101AC000CB027093CC028093CD029093CE020C9403
:101AD000510D0F931F936091CB027091CC028091B6
:101AE000CD029091CE028B019C0106701127222716
:101AF0003327063011052105310529F468601F914F
:101B00000F910C945F0D677FFACF0F931F9341E005
:101B100050E060E070E004C0440F551F661F771F5F
:101B20008A95D2F7CB01BA01609570958095909512
:101B30000091CB021091CC022091CD023091CE02C7
:101B400060237123822393231F910F910C945F0DC7
:101B500090915D028095892380935D02282F2770E4
:101B600039F4282F082E000C330B9217130621F49A
:101B700090916C0292FF07C08595859585950E948E
:101B8000850D10925D0208950F931F9341E050E080
:101B900060E070E004C0440F551F661F771F8A95F0
:101BA000D2F78091CB029091CC02A091CD02B0915E
:101BB000CE028A019B01082B192B2A2B3B2BC90132
:101BC000B8011F910F910C945F0D609362027093A6
:101BD000630280936402909365020C94510D8823F4
:101BE00041F08095909160028923809360020C946B
:101BF000E50C0895882339F090916002982B90931A
:101C000060020C94E50C0895882309F452C08238D0
:101C100071F40E94230981FF4CC089E30E947B0874
:101C20000E94E50C89E30E946E080C94E50C833851
:101C300059F40E94230980FF3CC083E50E947B0881
:101C40000E94E50C83E5EFCF843859F40E94230904
:101C500082FF2FC087E40E947B080E94E50C87E486
:101C6000E2CF9CEF980F913AF0F290E2980F983003
:101C700088F4877021E030E0A90102C0440F551FAD
:101C80008A95E2F7CA01809590916002892380933A
:101C90006002CBCF9BE5980F933020F490E080E07A
:101CA0000C940D09885A873120F490E080E00C9460
:101CB000F7080895CF93DF93D82FC0916C02C2FB31
:101CC000882780F98D17F9F0D0FBC2F9C0936C0218
:101CD00060916B0284E090E00E9416336C2F82E2E8
:101CE00090E00E94163380919B0280FF0CC01F92EF
:101CF000DF9388E598E09F938F930E94B8060F903A
:101D00000F900F900F90DF91CF910895109288025D
:101D10008091890284608093890280919B0280FF78
:101D200008C087E693E09F938F930E94B8060F90B8
:101D30000F9008959FB7F8941092AB029FBF9091B7
:101D4000BA02943009F048C02091E9002F70309118
:101D5000EC00932F917030FD90E8922B25E02093BA
:101D6000E9002091EB0020FF34C02091EE0027FF16
:101D700030C020916602222321F02091E80025FF47
:101D800028C01092660226E03091E80035FF14C0AA
:101D90008093F1008091E80085FD27C08091E800E4
:101DA00080FFFCCF8091E8008E778093E8009F70E1
:101DB0009093E90080E008953091BA02343049F4FC
:101DC0003091EB0035FD05C0215041F481E0809356
:101DD00066029F709093E9008FEF0895EFE9FFE0AE
:101DE0003197F1F700C00000CFCF8FB7F89421E012
:101DF0002093AB028FBFDBCFCF93DF9300D00F9246
:101E0000CDB7DEB79091BA02943011F589837B8308
:101E10006A839093E9008FEF9091E800815095FDDF
:101E200006C095ED9A95F1F700008111F5CF8091EC
:101E3000E80085FF0DC050E040E063E070E0CE01B7
:101E400001960E9411078091E8008E778093E80048
:101E50000F900F900F90DF91CF910895BC0184E017
:101E60000C94FC0EBC0183E00C94FC0ECF93DF932A
:101E7000EC0181E08093E9008FEF9091E8008150C0
:101E800095FD06C095ED9A95F1F700008111F5CF0B
:101E90008091E80085FF14C050E040E068E070E009
:101EA000CE010E9411078091E8008E778093E800B0
:101EB00088E0FE01A0EBB2E001900D928A95E1F777
:101EC000DF91CF91089581E08093E00080E28093DC
:101ED000D8001092C9008FE19EE40197F1F700C08D
:101EE000000087E090EBDC018093E7029093E8022A
:101EF000A093E902B093EA0288E19CE00FB6F8945F
:101F0000A895809360000FBE90936000FFCFCF93A1
:101F1000C82F882309F488C08238C1F40E9423099D
:101F200081FD82C089E30E947B080E94E50C2FEFAF
:101F300081EE94E0215080409040E1F700C0000025
:101F400089E30E946E08CF910C94E50C8338A1F4CC
:101F50000E94230980FD68C083E50E947B080E94DF
:101F6000E50C2FEF81EE94E0215080409040E1F7A6
:101F700000C0000083E5E5CF8438A1F40E94230966
:101F800082FD52C087E40E947B080E94E50C2FEF7F
:101F900081EE94E0215080409040E1F700C00000C5
:101FA00087E4CFCF8CEF8C0F813A68F4E6ECF1E058
:101FB0008191C81799F121E0EC3CF207C9F78C2F09
:101FC0000E947B08C0CF80E28C0F883068F4C77015
:101FD00021E030E001C0220FCA95EAF7809160024B
:101FE000822B80936002AFCFEBE5EC0FE33040F43F
:101FF000F0E0E459FE4F808190E0CF910C940D0900
:10200000C85AC73188F4EC2FF0E0EE0FFF1FE159FA
:10201000FE4F80819181CF910C94F7088C2F0E9404
:102020006E080E94E50CCBCFCF9108951F93CF93FC
:10203000DF93182FD0E0C0E0893311F4C0E5D0E081
:10204000812F0E94870F209731F4812FDF91CF914C
:102050001F910C94040E8FE99FE00197F1F700C0E7
:1020600000002197F0CF0F931F93CF93DF93C62FDC
:10207000D42F022FFC0182818823A1F06093CA0231
:102080000E945C089093C9028093C802C77081E0E7
:1020900001C0880FCA95EAF7DF91CF911F910F9188
:1020A0000C94FA0D8091CA02681340C02091C802B6
:1020B0003091C9024FB7F8948091C4029091C50243
:1020C000A091C602B091C7024FBF821B930B883C00
:1020D000910560F510E21D0F6D17B9F080E2860FD3
:1020E000883040F4C77081E001C0880FCA95EAF7D4
:1020F0000E94EF0D183048F481E09D2F977001C0C9
:10210000880F9A95EAF70E94FA0D802F0E94161008
:10211000183098F4D77081E001C0880FDA95EAF79B
:10212000DF91CF911F910F910C94EF0DC77081E05B
:1021300001C0880FCA95EAF7F3CFDF91CF911F91C5
:102140000F91089560910F0180919C0280FF20C043
:1021500080910E0143E0849FC00111248C529E4F58
:10216000569A2BB12F7B3BB130645FB7F894FC01DA
:10217000649FE00DF11D1124BF0168177907D1F4A8
:102180005FBF8FE594E00197F1F700C0000008956C
:10219000809110019091110123E0829FF0011124A0
:1021A000EC52FE4F8917A0F61182108212828F5FC7
:1021B0003396F8CFFC014191CF01E8E03BB9000034
:1021C00000C047FF2BB9440F000000C000C000C092
:1021D0002BB900C0EA9591F7D0CF0F931F93CF93FF
:1021E000DF93EC0110E000E09091120190171106CE
:1021F00009F06CF40E94A2108C8190E0019681702D
:1022000099278C83DF91CF911F910F910895209191
:102210001001A801420F511D9A01220F331F240FF4
:10222000351F2C523E4F4C8160919E0280919D0241
:1022300096959017110651F04CF0442349F04091C7
:102240009F020E9443090F5F1F4FCECF4423B9F373
:1022500040E0F7CFEF92FF921F93CF93DF93EC0113
:1022600010E0EE24EA94F12C60911201161770F040
:102270000E94A2109A818C8190FF27C08F5F8C836F
:10228000DF91CF911F91FF90EF9008952091100161
:10229000422F410F5527551FCA019A01220F331FA4
:1022A000280F391F2C523E4F70E0C7010E948E321A
:1022B000962F8C8140919F0260919E02199F800D04
:1022C00011240E9443091F5FCFCF8150D8CF8F9236
:1022D0009F92AF92BF92CF92DF92EF92FF920F93B5
:1022E0001F93CF93DF93EC018A81BB24BA9480FDC6
:1022F00002C0BB24B394A09012018C81811109C04B
:1023000081E0B81228C08FEF8A0D8093D10181E05F
:102310008C83F12CE12C4CE0942EEA14F8F00E940E
:10232000A2108091D10191E0B9125FC0811158C013
:102330008091120181508093D1011C82DF91CF9155
:102340001F910F91FF90EF90DF90CF90BF90AF90D3
:102350009F908F9008951092D101D9CF00911001D4
:102360000E0D1F2D111DC801880F991F080F191F71
:102370000C521E4FF80111821082128234E0C32EDB
:10238000D12C812C8091D101880D8D302CF1692DBB
:102390000E946C32892F082E000C990B8E159F0518
:1023A00091F480919F028C9DA0018D9D500D112470
:1023B0005595479555954795980160919E02809156
:1023C0009D020E9443098B0CF1E0CF1AD108D1F68F
:1023D0008FEFE81AF80AA1CF87FFDDCF8A0DDBCF98
:1023E00081508093D101BC82A9CF90E00196609189
:1023F000120170E00E948E328093D1018C839ECFB7
:10240000EF92FF920F931F93CF93DF93EC018C8198
:10241000811109C081E08C831092D20192E09093E7
:102420000C0180930B01809110019091110123E028
:10243000829FF0011124EC52FE4F891768F110E0E1
:1024400003E060911201161768F10E94A2108091BA
:102450000B012091D201280F2093D20190910C0101
:10246000980F90930C01191654F4022E000C330BA4
:10247000409112014150550B2417350734F08195D6
:1024800080930B01813009F41C82DF91CF911F9161
:102490000F91FF90EF9008951182108212828F5F4A
:1024A0003396CBCFE12EF12C70E0C7010E948E3223
:1024B00020911001820F482F50E02091D201022E6E
:1024C000000C330BE216F306BCF020910C01022E37
:1024D000000C330B2E153F057CF0809F90011124DA
:1024E0002C523E4F40919F0260919E0280919D022E
:1024F0000E9443091F5FA5CFFA01EE0FFF1FE40FF3
:10250000F51FEC52FE4F118210821282F3CF8F9290
:102510009F92AF92BF92CF92DF92EF92FF920F9372
:102520001F93CF93DF93EC014C81042F10E09801AF
:10253000D8010E94D9329B01AC010E94EF324B01BD
:102540005C01E0E2F0E0E01BF10BA5E5B0E0AC01DE
:102550009B010E94EF326B017C019F01DF010E9411
:10256000D1329B01AC010E94FA329B01AC01280DD3
:10257000391D4A1D5B1DC701B6010E94A232F22E11
:10258000822F90E039E23F1560F143E0249F9001F3
:10259000112435952795122F109500E085E5E82E3A
:1025A000EF1880911201081758F10E94A2109C8127
:1025B00081E0992319F0903219F48FEF80930D0187
:1025C00080910D01890F8C83DF91CF911F910F9125
:1025D000FF90EF90DF90CF90BF90AF909F908F9043
:1025E000089525E530E0B901681B790B9B01220FA6
:1025F000331F260F371F37FFCCCF2F5F3F4FC9CF79
:102600008E2D01FD8F2D20911001622F600F7727F5
:10261000771F9B01220F331F260F371F2C523E4F6F
:10262000412F60919E020E9443090F5FBACF9091A3
:102630009C0290FF14C0909110012091110133E091
:10264000939FF0011124EC52FE4F921710F00C945E
:10265000A2108183608342839F5F3396F6CF0895F3
:102660000F931F93CF93DF9300D00F92CDB7DEB7B8
:102670008C018091D30181110AC09E012F5F3F4FD1
:102680004FEF6FEF0E9443098A818093D301F801D5
:102690006481613069F08091D30140E0662361F08C
:1026A00040E0623011F44091D30180E060E004C06A
:1026B0006091D30140E080E00E941713F80184810B
:1026C00090E0019663E070E00E948E3284830F9068
:1026D0000F900F90DF91CF911F910F910895CF939D
:1026E000DF9300D00F92CDB7DEB790919C0290FFA0
:1026F0000AC09E012F5F3F4F0E9443094B816981B1
:102700008A810E9417130F900F900F90DF91CF9145
:102710000895CF93DF93EC01EC81F0E0E058FC4F9B
:102720004491ECE9F2E0628181810E946F138C8117
:102730008F5F8C83DF91CF910895CF93DF93EC016E
:10274000ECE9F2E0438162818C810E946F138C81FD
:102750008F5F8C83DF91CF91089580919C028E7F53
:1027600080939C0280919B0280FF0CC01F921F925D
:102770008CE992E09F938F930E94B8060F900F9080
:102780000F900F900E94860E809189028160809345
:1027900089022FEF80E792E0215080409040E1F7DE
:1027A00000C000000C94A2108091D001811110C0D3
:1027B0008091D80080618093D8008AE18A95F1F7F2
:1027C00000C08091D90080FF0AC081E08093D001D1
:1027D00081E09091D001913009F080E0089582E08D
:1027E0008093D0010E94C1061092BA02F1CF6AEE26
:1027F0007EEF90E080E00E94343360E082E090E081
:102800000E94163360E083E090E00E94163310923D
:10281000620210926302109264021092650260E0FC
:1028200084E090E00E94163360E082E290E00E9433
:10283000163360E085E090E00E94163360E086E0A9
:1028400090E00E9416336FEF87E090E00E9416330D
:1028500040E050E0BA0188E090E00E94283360E058
:102860008DE090E00E94163340E050E0BA0188E12C
:1028700090E00E94283360E087E190E00E941633E8
:1028800040E050E0BA018CE190E00E94283370E013
:1028900060E080E290E00E94343340E050E0BA0112
:1028A00088E190E00E94283340E050E0BA018FE0D8
:1028B00090E00E94283340E050E0BA0183E190E0CC
:1028C0000C942833CF92DF92EF92FF926B017C0140
:1028D0000E943409B701A60188E090E0FF90EF90D4
:1028E000DF90CF900C9428334F925F926F927F923B
:1028F0008F929F92AF92BF92CF92DF92EF92FF9210
:102900000F931F93CF93DF9300D00F92CDB7DEB715
:10291000182FF62E042F722E90919C0290FF57C014
:10292000E92FE695AE2FB0E0A95BBE4F8C91809366
:1029300087029E7F923009F05EC09E012F5F3F4F5D
:10294000812F0E9443094B8169818A810E9417135C
:1029500080919D02811308C080919E028F1104C056
:1029600080919F02801729F0809189028260809374
:10297000890210939D02F0929E0200939F0277209D
:1029800009F49CC060919C0270919D0280919E020E
:1029900090919F020E94621480919B0280FF17C059
:1029A00080919F021F928F9380919E021F928F931E
:1029B00080919D021F928F938DEF92E09F938F9352
:1029C0000E94B8060FB6F894DEBF0FBECDBF0F90C1
:1029D0000F900F90DF91CF911F910F91FF90EF908B
:1029E000DF90CF90BF90AF909F908F907F906F902F
:1029F0005F904F900895823019F400919F02A8CF04
:102A0000863019F410919D02A3CF8930D9F3893112
:102A100009F09ECFE9518E2F8170682E8E2F809500
:102A20008170E82EE695F0E0E75BFC4FC590D4900E
:102A3000412CDD2492E2A92E93E0B92E609112017F
:102A4000461618F00E94A21083CF842C912C8C9CE7
:102A5000C0018D9C900D9C9C900D112470E00E94F3
:102A60007A32512E611028C0560E80919B0280FF51
:102A700011C0DF92CF921F92EF921F925F921F922E
:102A80004F92BF92AF920E94B8060FB6F894DEBF85
:102A90000FBECDBF20911001820E911C9401220F18
:102AA000331F280D391D2C523E4F402F6F2D852D81
:102AB0000E9443094394C2CF561AD7CF80919B02FC
:102AC00080FF85CF1F920F931F92FF921F921F933B
:102AD00086ED92E073CFECE9F2E0438121E1421B05
:102AE00008F440E021E0628181810C947414ECE9E7
:102AF000F2E0438121E1420F08F44FEF21E06281CF
:102B000081810C947414ECE9F2E0628121E1621B92
:102B100008F460E021E0438181810C947414ECE9B5
:102B2000F2E0628121E1620F08F46FEF21E043815E
:102B300081810C947414ECE9F2E0818121E04381FD
:102B4000628188500C947414ECE9F2E0818121E0F8
:102B500043816281885F0C9474148091A002882361
:102B600019F081508093A00260919C0270919D02A7
:102B700080919E0290919F020C9462148091A00219
:102B8000833018F48F5F8093A00260919C02709153
:102B90009D0280919E0290919F020C946214ECE938
:102BA000F2E087E1808311828FEF828380E8838364
:102BB0001482A7E8B2E012968C9112978360129665
:102BC0008C9360817181828193810C946214109244
:102BD0006002E6ECF1E086E0DF011D928A95E9F7FC
:102BE0000C94510D1F93CF93DF93CDB7DEB7AA9707
:102BF0000FB6F894DEBF0FBECDBF8CEB92E02091F4
:102C0000F100DC012D93CD01B2E0843C9B07B9F7C4
:102C10008091BD02833009F471C0B8F4813009F4A9
:102C200048C0823009F4B2C08091E80083FF3AC105
:102C30008091BC029091BD029A3008F033C1E92F17
:102C4000F0E0E959FC4C0C94C4328A3009F48DC090
:102C50008B3009F470C0893039F78091BC02813221
:102C600019F78091C0029091C102009711F002976C
:102C7000D9F68091E800877F8093E8008091E80092
:102C800082FF37C09091F3008091F200029729F4FF
:102C90008091F1008B7F813021F48091F10080934D
:102CA000AF028091E8008B778093E8000E943B0799
:102CB000BBCF8091BC02813A09F0B6CF8091E80089
:102CC000877F8093E8008091C0029091C102892B98
:102CD00061F468E080EB92E070E00E94ED07809183
:102CE000E8008B778093E8009FCF60E090E080E081
:102CF000F3CF8091BA028111C1CF96CF8091BC02EF
:102D0000813A09F091CF8091C0029091C102892B44
:102D100009F08ACF8091E800877F8093E800809156
:102D2000E80080FFFCCF809130018093F10080911A
:102D3000E8008E77B9CF8091BC02813209F074CF60
:102D40008091C0029091C102892B09F06DCF8091D2
:102D5000E800877F8093E8000E943B078091BE02D5
:102D6000809330010E94E7155FCF8091BC028132D1
:102D700009F05ACF8091E800877F8093E8000E9495
:102D80003B078091BF028093AE024ECF8091BC0280
:102D9000813A09F049CF8091E800877F8093E8006D
:102DA0008091E80080FFFCCF8091AE02BECF8038DA
:102DB00099F0823809F076C08091C0028F70873018
:102DC00008F070C08093E9008091EB0085FB8827B4
:102DD00080F91092E90006C08091B8029091B90282
:102DE000911182609091E800977F9093E800809322
:102DF000F1001092F1008091E8008E77BAC188232B
:102E000009F4A7C1823009F04DC08091BE02811142
:102E1000ABC18091C0028F702FEF280F263008F0D1
:102E200041C08093E9002091EB0020FF9DC19330C9
:102E300031F48091EB0080628093EB0095C190911A
:102E4000EB0090619093EB0021E030E001C0220F95
:102E50008A95EAF72093EA001092EA008091EB004D
:102E60008860EACF81111EC01091BE021F77809149
:102E7000E3008078812B8093E3008091E800877FD6
:102E80008093E8000E943B078091E80080FFFCCF20
:102E90008091E30080688093E30082E0111183E079
:102EA0008093BA028091E80083FF0AC08091E80015
:102EB000877F8093E8008091EB0080628093EB0035
:102EC000AA960FB6F894DEBF0FBECDBFDF91CF91AB
:102ED0001F9108958058823028F72091BE023091CA
:102EE000BF022C3DE3E03E07A1F583E08A838AE23E
:102EF00089834FB7F894DE01139620E03EE051E25B
:102F0000E32FF0E050935700E49120FF03C0E295D7
:102F1000EF703F5FEF708E2F90E0EA30C0F0C79601
:102F20008D939D932F5F243159F74FBF8091E80017
:102F3000877F8093E8006AE270E0CE0101960E94EC
:102F4000ED078091E8008B778093E800ABCFC096C7
:102F5000E7CF8091C0029091C102432F55274330A3
:102F6000510509F44AC078F54130510509F47AC099
:102F70008BE790E0E8EDFAE04230510509F092CF9E
:102F80002091E800277F2093E8002091C202309131
:102F9000C3028217930708F49C0140E02115310514
:102FA00009F065C0411163C08091E80082FDC9CF7E
:102FB0008091BA02882329F2853019F28091E800C5
:102FC00083FFF2CFBECF4132510509F43CC04232FB
:102FD000510509F067CF8430910508F063CFFC01FB
:102FE000EE0FFF1FEF54FE4F0190F081E02D83554F
:102FF0009E4FDC018C9190E01AC0332721303105BF
:10300000D1F02115310561F02230310509F04ACFA8
:10301000E5E6FBE0E4918E2F90E0E5E6FBE007C0FB
:10302000EFE8FBE0E4918E2F90E0EFE8FBE0009703
:1030300009F438CFA5CFEFE7FBE0E4918E2F90E0C5
:10304000EFE7FBE0F4CF8430910508F02BCF880F39
:10305000991FFC01E754FE4F0190F081E02D89E0BB
:1030600090E08ECF82E190E0E3E5FBE089CF8091B4
:10307000BA02882309F465CF853009F462CF8091C4
:10308000E80083FD5ECF8091E80082FD8DCF8091C6
:10309000E80080FF83CF9091F3008091F20021152A
:1030A000310519F08830910550F041E0089709F09A
:1030B00040E08091E8008E778093E8006FCF4491E4
:1030C0004093F1003196215031090196E8CF8038C4
:1030D00009F0E8CE8091E800877F8093E800809136
:1030E000BB028093F10087CE8111DCCE1091BE022D
:1030F000123008F0D7CE8091E800877F8093E800F7
:103100001093BB020E943B07112311F084E005C01D
:103110008091E30087FDFACF81E08093BA0242E01C
:1031200061EC81E00E945A0742E261EC84E00E9477
:103130005A0742E261EC82E00E945A0742E260ECE8
:1031400083E00E945A0742E261EC85E00E945A0740
:10315000A9CE8091BE02813009F0A4CE81E09330E7
:1031600009F080E08093B9021092E9008091E800B4
:10317000877F8093E8000E943B0794CE8F929F92B6
:10318000AF92BF92CF92DF92EF92FF920F931F9375
:10319000CF93DF9300D000D00F92CDB7DEB709E117
:1031A00011E08DE6C82E82E0D82E4601F12CAA242B
:1031B000A394B12CD8018D918D01F894E82FE2955C
:1031C000EF70F0E021A18F70A50102C0440F551FE0
:1031D0008A95E2F7CA01922F982B91A392A180952C
:1031E000892382A3789400C0E3E1F1E030E020E09D
:1031F000E12C4191A42FA295AF70B0E090968C91F4
:1032000090E04F7002C0959587954A95E2F780FD52
:1032100053C08A2D022E01C0880F0A94EAF7E82ACB
:103220002F5F3F4F2630310521F7F801319780811C
:103230000E94D90950EA5A95F1F7D4018C91E81609
:10324000E9F1EC9281E0F82ABFEF8B1A9B0AE1E0EA
:103250000E311E0709F0AECF10917802FF2081F1E8
:1032600081E08093CE010E945C089093CD01809311
:10327000CC012091CC013091CD014FB7F8948091D1
:10328000C4029091C502A091C602B091C7024FBF7F
:10329000821B930B0697C0F0E12FF0E0EF55FD4F36
:1032A000D6018D916D018193B2E7CB16B2E0DB06BA
:1032B000B9F71092CE0108C080E0B1CF80E0C3CF53
:1032C0008091CE018111D5CF0E94D413E82E609158
:1032D0007802882309F455C08E010F5F1F4F85E0E7
:1032E000F80111928A95E9F7862F90E0B8018F5581
:1032F0009D4F0E942F30811127C08091CF018F5F99
:103300008093CF018630D8F1E0917702F0E0EF555D
:10331000FD4F10821182128213821482F11001C0BB
:10332000FE2C8F2D0F900F900F900F900F90DF912C
:10333000CF911F910F91FF90EF90DF90CF90BF90B2
:10334000AF909F908F9008951092CF01A091770237
:10335000B0E0AF55BD4F9E012A5F3F4FE12C4D912C
:10336000F80191918F01491731F0AD014150510998
:10337000FA019083E82E0217130789F7CFCFE12CCB
:10338000CDCF70E06F557D4F8091770290E08F55E3
:103390009D4F0E946830C2CF1F920F920FB60F92BE
:1033A00011242F933F934F935F936F937F938F934A
:1033B0009F93AF93BF93CF93DF93EF93FF93D091FE
:1033C000E900DF708091EC00C82FC17080FDC0E87B
:1033D0001092E9008091F000877F8093F00078944C
:1033E0000E94F2151092E9008091F00088608093AD
:1033F000F000CD2BCF70C093E900FF91EF91DF91EA
:10340000CF91BF91AF919F918F917F916F915F917C
:103410004F913F912F910F900FBE0F901F901895D5
:103420001F920F920FB60F9211242F933F934F9339
:103430005F936F937F938F939F93AF93BF93EF931C
:10344000FF938091E10082FF15C08091E20082FF2E
:1034500011C08091E1008B7F8093E1002091AC024C
:103460002F5F822F62E30E946032992309F4BEC06D
:103470002093AC028091DA0080FF28C08091D800B0
:1034800080FF24C08091DA008E7F8093DA008091E3
:10349000D90080FFE1C080E189BD82E189BD09B426
:1034A00000FEFDCF81E08093BA0284EC9AE00E9496
:1034B0001F068091AD02811109C00E94C1060E94C1
:1034C0008C078091E20084608093E2008091E100AB
:1034D00080FF1BC08091E20080FF17C08091E20056
:1034E0008E7F8093E2008091E20080618093E20011
:1034F0008091D80080628093D80019BC85E08093C9
:10350000BA028CEC9AE00E941F068091E10084FFD1
:103510002DC08091E20084FF29C080E189BD82E155
:1035200089BD89B5982F917080FFFBCF8091D8001D
:103530008F7D8093D8008091E1008F7E8093E100A1
:103540008091E2008F7E8093E2008091E2008160B2
:103550008093E2008091BB02882309F487C084E055
:103560008093BA0280ED9AE00E941F068091E100EC
:1035700083FF2BC08091E20083FF27C08091E10090
:10358000877F8093E10082E08093BA021092BB02B1
:103590008091E1008E7F8093E1008091E2008E7F38
:1035A0008093E2008091E20080618093E20042E03B
:1035B00060E080E00E945A078091F000886080936C
:1035C000F00084ED9AE00E941F06FF91EF91BF91F9
:1035D000AF919F918F917F916F915F914F913F91AB
:1035E0002F910F900FBE0F901F9018951092AC0264
:1035F0008091AB02882309F43DCF8091BA028430D8
:10360000C1F49091E9009F702091EC00822F8170AD
:1036100020FD80E8892B95E09093E9009091EB00E4
:1036200090FF04C09091EE0097FD08C08F708093CA
:10363000E9001092AB021ECF1092F1009091E800C9
:1036400095FDFACF9091E80090FFF0CF9091E800BF
:103650009E779093E800EACF19BC1092BA0288ECEA
:103660009AE00E941F061092AD0230CF8091E300D5
:1036700087FD93E09093BA0275CF80919A02869568
:103680008695869508950F931F930E94D4138823DF
:1036900021F01F910F910C9450080E945008009146
:1036A0006702109168022091690230916A02600FEE
:1036B000711F821F931F1F910F9108950E94D413B1
:1036C00081110C945C080E94431BCB01089560910A
:1036D0009C02669570E04BE050E080E091E00E9433
:1036E0004A33892B19F481E0809388020E945E1B83
:1036F00090938202809381028091890284608093FA
:10370000890280919B0280FF08C08EE493E09F9322
:103710008F930E94B8060F900F90089590919C028D
:1037200090FF5AC09170811141C0926090939C02A9
:10373000809189028160809389026623F1F1609112
:103740009C0270919D0280919E0290919F020E9426
:10375000621480919B0280FF0FC080919C0286952D
:103760001F928F9380E892E09F938F930E94B806F8
:103770000F900F900F900F9060919C02669570E0F3
:103780004BE050E080E091E00E944A33892B09F140
:103790000E94860E81E08093840220E040919F0287
:1037A00060919E0280919D020C947414853210F0F9
:1037B0009864BCCF880F982BB9CF80919B0280FF73
:1037C000DBCF80919C0286951F928F9382E692E0D8
:1037D000CBCF0E94671BDECF089580919C02869517
:1037E000815009F484E261E00C948E1B80919C026C
:1037F00086958F5F853208F081E061E00C948E1B26
:1038000090919C0290FF07C09695981720F096170C
:1038100010F40C94F61B61E00C948E1BCF92DF9297
:10382000EF92FF926B017C010E94D41381110EC0B4
:103830000E945008C61AD70AE80AF90AC09267021D
:10384000D0926802E0926902F0926A02FF90EF90D3
:10385000DF90CF90089578941F921FB61F92112485
:103860008F939F93AF93BF938091C4029091C502B1
:10387000A091C602B091C7020196A11DB11D80930F
:10388000C4029093C502A093C602B093C702BF9131
:10389000AF919F918F911F901FBE1F9018951F92FF
:1038A0001FB61F9211248F939F93AF93BF93809164
:1038B0007D02811113C08091C4029091C502A09134
:1038C000C602B091C7024196A11DB11D8093C402EA
:1038D0009093C502A093C602B093C702BF91AF9167
:1038E0009F918F911F901FBE1F901895FF920F936D
:1038F0001F93CF93DF93D0917A020D2F10E00657DC
:103900001D4FFC01C081F8018081C81BFC2E80E0A6
:103910001F147CF09C2FC7FD90E0C91BC11118C07B
:10392000882329F1DF91CF911F910F91FF900C9483
:10393000F508FA94F80180818F5F80838AEADD239D
:1039400019F0D13019F48BE40E94161081E0E0CF19
:10395000CF5FF80180818150808389EADD2319F0EF
:10396000D13019F48EE40E94161081E0D7CFDF9198
:10397000CF911F910F91FF900895E0918D02F0E09B
:10398000E657FD4F2081FC0120830895CF92DF92FE
:10399000EF92FF92863030F5811125C09091800022
:1039A0009F77909380002D98282F30E0AFEFBFEFE6
:1039B0000E94D93225E030E040E050E00E94A2327F
:1039C000C9012C3764E13607A0F469E070E00E9479
:1039D0007A327093890060938800FF90EF90DF90B7
:1039E000CF90089585E0909180009068909380003A
:1039F000DBCF2A50374D4F4F5F4F942F832F722FBD
:103A0000662725EF38E241E050E00E94A2326901CA
:103A10007A01CA01B9010E9450329B01AC01C70171
:103A2000B6010E945032672F782F892F9927611590
:103A3000710521E08207910561F66FEF7FEFC9CF35
:103A4000282F220F220F220F90919A029770922B0B
:103A500090939A02987F21E009F420E090919A02D5
:103A600020FB90F990939A020C94C61C3F924F92BF
:103A70005F926F927F928F929F92AF92BF92CF92FE
:103A8000DF92EF92FF920F931F93CF93DF9300D0BB
:103A900000D00F92CDB7DEB78C01FC0183819481F9
:103AA000892B31F08081918189238F3F09F004C7F0
:103AB0000F900F900F900F900F90DF91CF911F916B
:103AC0000F91FF90EF90DF90CF90BF90AF909F90BD
:103AD0008F907F906F905F904F903F9008950E94DD
:103AE0000B0CF82E682F89819A810E94BD0869818C
:103AF0007A818F2D0E947F0A7C01F80182818823C0
:103B000009F4ADC6C70182519F45409708F01CC615
:103B10008FEF93E00E940233FEEEEF0E57E0852E0A
:103B200052E0952E882381F180915D02877009F41F
:103B3000BFCFF8018281882309F4BACF82E00F90C9
:103B40000F900F900F900F90DF91CF911F910F91D9
:103B5000FF90EF90DF90CF90BF90AF909F908F90AD
:103B60007F906F905F904F903F900C94A80D8114C0
:103B700024E09206C9F2C4010E940233811101C0FF
:103B8000EA943FEF831A930AE110F1CF1C821B8263
:103B9000442443944AE0342E74018FEFE81AF80A63
:103BA000C4010E94023389831A82882309F4BCCF9E
:103BB0009FEF980F933000F58A83498292E0890E37
:103BC000911CC7010E9402338B83882309F4ACCF78
:103BD000FE0131967F01F70120812223E9F2213095
:103BE00009F049C091818281913041F4F2E0EF0EF9
:103BF000F11C0E94161009C04701EACF923049F427
:103C000022E0E20EF11C0E94870F3FEFE31AF30A55
:103C1000E2CF933031F432E0E30EF11C0E94040E47
:103C2000F4CF943021F08FEFE81AF80AEECF92E04B
:103C3000E90EF11C30E020E0B7016F5F7F4FF70124
:103C400041818053990B8A30910550F02150310900
:103C5000E0F28FE99FE00197F1F700C00000F6CF96
:103C6000329EF001339EF00D11249C012E0F3F1F58
:103C7000842F7B01E1CFE22FF0E0E057F94F549021
:103C8000822F86958695869590E0FC01E058F94F45
:103C900064902770712C022E02C0759467940A9468
:103CA000E2F7E1E06E227724FC01E059F94FA4909D
:103CB000B12C022E02C0B594A7940A94E2F7F1E069
:103CC000AF22BB24FC01E05AF94FC490D12C02C0B2
:103CD000D594C7942A95E2F721E0C222DD2461142D
:103CE000710419F081EE0E94870FA114B10419F03C
:103CF00086EE0E94870F852D0E941610AB2819F0C2
:103D000086EE0E94040E672819F081EE0E94040ED0
:103D1000CD2809F47ACF8CE26CCF81E00E94C40DEB
:103D20000E94690D01CF81E00E94850DF9CF82E0EC
:103D3000F5CF82E0F9CF2FEBE2162CE5F20609F47D
:103D40008DC008F466C080ECE8168CE5F80609F032
:103D50001CC590919A02892F8695869586958F5FCE
:103D60008F719770863008F0ACC0880F880F880F6D
:103D7000892B80939A0280919A02887F91E009F4BE
:103D800090E080919A0290FB80F980939A020E94C1
:103D9000E00C80919B0280FFBEC580919A028695BF
:103DA000869586951F928F938BE797E029C085E0D3
:103DB0000E94201D80919A020E94E00CB5CE809155
:103DC0009A02982F987F79F0885080939A02887F82
:103DD00091E009F490E080919A0290FB80F9809341
:103DE0009A020E94E00C80919B0280FF94C5809112
:103DF0009A028695869586951F928F9380E197E02B
:103E00009F938F930E94B8060F900F900F900F9082
:103E100082C580919A02982F9695969596959530A1
:103E200040F49F5F990F990F990F8770892B8093AA
:103E30009A0280919A02816080939A020E94E00C1B
:103E400080919B0280FF67C580919A028695869536
:103E500086951F928F9388E297E0D2CFF0909A02D6
:103E6000F0FAFF24F0F880919B0280FF36C51F9284
:103E7000FF9285E697E09F938F930E94B8060F907C
